:020000040000FA
:06000000D23001303A2865
:08000800A000030EA100831209
:100010008B1C32288B1031181428B11C3228643004
:10002000010203183128182800001628172818285C
:1000300019281A281B281C281D281E281F283110A3
:10004000B114A810031005190314AA0DA90DA80DC9
:10005000B00B322831152A08AF002908AE00280855
:10006000AD00B11081010B11210E8300A00E200EF6
:02007000090085
:0C007400203084008001840A80300402E7
:10008000031C3C281230B0006B21850187018316C8
:100090000C30850587018312831605148715071612
:1000A0008312850187010730990000309A001030D3
:1000B00083168E008312603083168F008312003007
:1000C000831691009F008312C8308316810083122B
:1000D00031309000003083168C00831210308B007A
:1000E000BC1B7428851D0027D42181018E018F013E
:1000F0000B118B100B108C018B178C203119A22047
:10010000B30B8A28031085190314B90DF030390296
:100110000319F820C0237D286400311808000B1D46
:1001200008000B11B11031141230B000051D9D28CC
:10013000321483160113831208003210831601173C
:100140008312080031110130B7008B1320303707BC
:1001500083169B001C141A088312A400A500C0304B
:10016000A5061030370783169B001C141A0883124B
:10017000A3000030370783169B001C141A08831253
:10018000A2008B17321CCA2822090339A200A30936
:10019000A409A50922082D02031DF22823082E0216
:1001A000031DF22824082F02031DF2280130370214
:1001B000031DDD283D143E14B42102303702031D17
:1001C000E428BD143E14B82103303702031DEB2888
:1001D0003D153E14BC2104303702031DF228BD1525
:1001E0003E14C021B70A0530370203180800A528BD
:1001F0003C1C08000130B600B300B400B500B700E5
:1002000085018701B1138C20B30B1C2903108519BC
:100210000314B90DF030390203194329B41F071034
:10022000B40B1C293708B6080319B60003191A299C
:100230000714B6039630B400311D03293111321C66
:1002400026292D090339AD00AE09AF092F1CB113C2
:100250002F1C0329B11B03292E180329B1178B1357
:1002600020303707BB002F08BA005621103037075F
:10027000BB002E08BA00562100303707BB002D08FE
:10028000BA0056218B1785018701B70AB6010530E0
:100290003702031C0329D42108003E1C08003E102D
:1002A0001030BB003D08BA00562108008B133A08F5
:1002B00083161C159A0083123B0883169B00553049
:1002C0009D00AA309D009C1464009C1864291C1198
:1002D00083128B170800831600309B001C141A0829
:1002E0008312BC00831610309B001C141A08831262
:1002F000BD00831630309B001C141A088312D300F3
:1003000000309500603084008B13831604089B0036
:100310001C141A0883128B178000840A68300402A8
:10032000031C84296430D5004A24DC003C30EC00F6
:10033000ED00EE00EF00EA146E30D5004A240F39CC
:10034000031D08004F240F39031D080054240F39E2
:10035000031D080059240F39031D08008316871157
:1003600007128312EA1008000130E800E3210800B8
:100370000230E800E32108000430E800E32108002F
:100380000830E800E32108001030E800E32108000D
:100390002030E800E32108004030E800E3210800B5
:1003A0008030E800E3210800EA178B1383167030D1
:1003B0009B001C141A0883128B17E800E3210430F9
:1003C000EB00EA130800E80803190800681CF0298C
:1003D0006730D5004A24D1006830D5004A24D200C5
:1003E000E81CFA296730D5004F24D1006830D500C9
:1003F0004F24D200681D042A6730D5005424D10050
:100400006830D5005424D200E81D0E2A6730D5008C
:100410005924D1006830D5005924D200681E182A0A
:100420006A30D5004A24D1006B30D5004A24D2006E
:10043000E81E222A6A30D5004F24D1006B30D50047
:100440004F24D200681F2C2A6A30D5005424D100D2
:100450006B30D5005424D200E81F362A6A30D5000C
:100460005924D1006B30D5005924D200EA16D11A94
:10047000462A511B462A511C462ADC1FEA125C1FE1
:10048000462A501C462AC01B462A0800EA1E562A45
:10049000EA1B562A511870308B1383169B001C14CC
:1004A0001A0883128B17680203190800D11A612AEF
:1004B000511B612A6A10511C612A5014051E6A14CE
:1004C0000516511C692A511A5016D11AC017511B12
:1004D0005012EA1F702AD11A0800511B0800742A12
:1004E000D11AA12A511BA12A6530D500521A4A24DB
:1004F000D21A4F24521B5424D21B59245118C40021
:100500006630D500521A4A24D21A4F24521B542462
:10051000D21B59245118CC0052085118D70004306E
:100520006A183230EA1B32305118C80051185C1476
:10053000EA1F9F2A511C9E2A4403C000080051183C
:10054000C00151187030BB006808E900BA0056219C
:10055000BD010800FD010730FF007B08FE0C0318F9
:10056000B52AFF0BAE2AFB0100340310BA2AFE0C99
:100570000318FB07FB0CFD0CFF0BB72AFB0CFD0C53
:10058000003494019301093095008B138E018F0183
:100590008B17D6135608FB007508F51BFF3CFE00B1
:1005A000FE13AA22FD0D7B0DF51FD607F51BD60203
:1005B00056087607930003181414083095000800B5
:1007800002300F02031C0800EA1CED2BA1277108A0
:1007900003390319DA2B6E30D50071184A24F11889
:1007A0004F24E8006818B421E818B8216819BC2162
:1007B000E819C02171080C390319ED2B6E30D500F2
:1007C00071195424F1195924E8006818B421E81863
:1007D000B8216819BC21E819C0210730EB050330A6
:1007E0008A006B088207F82B352C362C372C382CD6
:1007F000501C432C4008D500571A4A24D71A4F24BE
:10080000571B5424D71B5924D600530856020318EB
:100810000715031C07116108F5006008F6005C1C51
:10082000C122C80B432C4C085C180530C8005C1C66
:10083000C00A5C1044084002031C432CC01B242C3B
:10084000501E242CC001432C7A182B2C7A1409300A
:10085000C800C003432C5012DC1805125C1950105C
:100860005C1DC0035C1DC017432C432C432C432C40
:10087000071C3C2C0710432CE9080319432C0714D0
:100880000310E90C432CEB0A05306B020318EB0153
:100890008F01080005308A00D51355088200053005
:1008A0008A00D5175508820006308A00D5135508EE
:0C08B000820006308A00D517550882002F
:100A00000034013403340434053406340834093422
:100A10000A340B340D340E340F34113412341334C1
:100A2000143416341734183419341B341C341D3460
:100A30001E342034213422342434253426342734FF
:100A400029342A342B342C342E342F34303432349D
:100A50003334343435343734383439343A343C343C
:100A60003D343E34403441344234433445344634DA
:100A7000473448344A344B344C344D344F3450347A
:100A800051345334543455345634583459345A3418
:100A90005B345D345E345F346134623463346434B7
:100AA00066346734683469346B346C346D346E3456
:100AB00070347134723474347534763478347A34F2
:100AC0007B347D347F347F34C43464340134013466
:100AD0001134003401341134003400340134003452
:100AE0000034003400340034003400340034003466
:100AF0000034003400340034003400340034003456
:100B00007F347E347C347B347A3479347734763471
:100B1000753474347234713470346E346D346C34B2
:100B20006B346934683467346634643463346234F3
:100B300061345F345E345D345B345A345934583434
:100B40005634553454345334513450344F344D3476
:100B50004C344B344A3448344734463445344334B7
:100B6000423441343F343E343D343C343A343934F9
:100B700038343734353434343334323430342F3439
:100B80002E342C342B342A3429342734263425347B
:100B900024342234213420341E341D341C341B34BC
:100BA00019341834173416341434133412341134FD
:100BB0000F340E340D340B340A3409340634053442
:100BC0000434033401340034C43464340134013453
:100BD0002234003401342234003400340034003430
:100BE0000034003400340034003400340034003465
:100BF0000034003400340034003400340034003455
:100C000080340034003401340234033404340634B4
:100C100008340A340C340E341134143417341A34B2
:100C20001D342134243428342C342F3433343734D5
:100C30003B343F34433447344B344F3452345634CE
:100C40005A345D346134643467346A346D347034DA
:100C500072347434763478347A347B347C347D3432
:100C60007E347E347E347E347E347D347C347B34FA
:100C70007A34783476347434723470346D346A343F
:100C80006734643461345D345A34563452344F34EA
:100C90004B34473443343F343B34373433342F34CC
:100CA0002C342834243421341D341A3417341434A9
:100CB00011340E340C340A3408340634043403344A
:100CC0000234013400340034C43464340134113447
:100CD00044340034013444340034003402340034E9
:100CE0000034003400340034003400340034003464
:100CF0000034003400340034003400340034003454
:100D000080340034003401340234033404340634B3
:100D100008340A340C340E341134143417341A34B1
:100D20001D342134243428342C342F3433343734D4
:100D30003B343F34433447344B344F3452345634CD
:100D40005A345D346134643467346A346D347034D9
:100D500072347434763478347A347B347C347D3431
:100D60007E347E347E347E347E347D347C347B34F9
:100D70007A34783476347434723470346D346A343E
:100D80006734643461345D345A34563452344F34E9
:100D90004B34473443343F343B34373433342F34CB
:100DA0002C342834243421341D341A3417341434A8
:100DB00011340E340C340A34083406340434033449
:100DC0000234013400340034C43464340134413416
:100DD0008834003401348834003400340034003462
:100DE0000034003400340034003400340034003463
:100DF0000034003400340034003400340034003453
:100E00003C1C08006C146D14EB011430B600071084
:100E10000130EB0507308A006B088207102F172F6F
:100E20006108F5006008F6000516D6011A2F7F301C
:100E3000D6001A2F701A432F6B18232F7019F60A39
:100E40007018F603272F7019F50A7018F503503043
:100E50007018EC007019ED00C8307602C830031825
:100E6000F600503076025030031CF600F51F3E2F7E
:100E7000873075028730031CF500432F64307502FC
:100E800064300318F5007F30D6006B1CD601C122F8
:100E9000EA017927701C4E2F6D1B7016701D522FA2
:100EA0006C1B7016701E572FEB0A6B1C682F0710F7
:100EB000B60B5F2F07143C306B180A30B600640085
:100EC0000A300F02031C5F2F8F01701A082F1A2F90
:100ED0007508E1007608E000603084000408BB007B
:100EE0000008BA005621840A68300402031C6E2FE1
:100EF0000800F0010A30851DEC078519EC027830F6
:100F00006C020319701479300318EC0015306C0270
:100F10000319F0141430031CEC000A30051CED0713
:100F20000518ED0278306D02031970157930031839
:100F3000ED0015306D020319F0151430031CED009F
:100F40000800F10114308719EE070230871DEE0208
:100F5000EE1BB52F14306E020318BE2F1430EE00B6
:100F6000F21CF114F2147210BE2F721C7114721460
:100F7000F2106E1BBC2FBE2FC030EE001430071ACB
:100F8000EF070230071EEF02EF1BD12F14306F0264
:100F90000318DA2F1430EF00F21DF115F21572115B
:100FA000DA2F721D71157215F2116F1BD82FDA2FFF
:060FB000C030EF00080054
:084000000A00030006000200A3
:02400E00CC33B1
:10420000010003000300030003000200020002009B
:1042100002000000000000000000FF00FF00FF009F
:10422000000000000000000000000000000000008E
:104230000000C000C000C000C000FF00FF00FF0081
:104240000100C300F300CF00FF00C300F300CF0064
:10425000FF00C300F300CF00FF00FF00FF00FF00DE
:104260004000FF00FF00FF00FF00FF00FF00FF0015
:10427000FF00FF00FF00FF00FF00FF00FF00FF0046
:10428000FF00FF00FF00FF00FF00FF00FF00FF0036
:10429000FF00FF00FF00FF00FF00FF00FF00FF0026
:1042A000FF00FF00FF00FF00FF00FF00FF00FF0016
:1042B000FF00FF00FF00FF00FF00FF00FF00FF0006
:1042C0007D00D4007D00D4007D00D4007D00D400AA
:1042D000FF00FF00FF00FF00FF00FF00FF00FF00E6
:1042E0000000000000000000FF00FF00FF00FF00D2
:1042F000FF00FF00FF00FF00FF00FF00FF00AA001B
:00000001FF
